:10494D000000090101240200000301FA0400FA0528
:10495D0000020A0A5A0B000F0C00FA0D00030E009C
:10496D00030F0132100096120132130AFA140102DC
:10497D0015000217010A18010A1905321A010A1B3E
:10498D00010A1C053223011E2400642A00FA2B00A3
:10499D00FA2C50782D003C2E00462F001E3000645E
:1049AD003250783300003432FA3501643601643701
:1049BD000150380A643C00643E003C3F000140FF5A
:1049CD00FF411450420A5A430AC844053245007843
:1049DD004600FA4701224802034C00FA4EFFFF50F1
:1049ED000404510596521432530B28540A9656025C
:1049FD0002570546580002590A465A32FA5B010A17
:104A0D005C14325E000A5F00FE61FFFF64021067F6
:104A1D0001036A0A3C6B00006C3296780132790111
:104A2D0032FAFAFA0065006F00790083008D009765
:104A3D0000A100AC00B600C000CA00D400DE00E842
:104A4D0000F2005B0063006A0072007A0082008948
:104A5D000091009900A100A800B000B800BF00C7E8
:104A6D0000CF00D600DF00E600EE00F60040004665
:104A7D00004C00520059005F0065006B007100771B
:104A8D00007D00830089008F0095009C00A200A886
:104A9D0000AE00B400BA00C000C600CC00D200D9F0
:084AAD0000DF00E500EB00F161
:10009E00AE32AF33740A8E048F05FF1200858C3496
:1000AE008D35AE32AF33740A8E048F05FF124BCEF0
:1000BE008C328D33E53345326013740AC39533FFAA
:1000CE00E49532FE8E328F337834124C1AE54FA8F7
:1000DE0034B80015D395354010E54FC39535FFE480
:1000EE009534FE8E348F358010E54F2424C395351C
:1000FE00FFE49534FE8E348F35754F00AE34AF3538
:10010E0074116F4E600674126F4E7018AE34AF35A8
:10011E0074116F4E7005754F018003754F02753562
:10012E0010753400AE34AF3574146F4E600674150E
:10013E006F4E7018AE34AF3574146F4E7005754F28
:10014E00018003754F02753513753400AE34AF352B
:10015E0074236F4E600674246F4E7018AE34AF3534
:10016E0074236F4E7005754F018003754F02753500
:10017E002275340022900079E0B40104C20B800293
:10018E00D20B90007AE0B40104C20C8002D20C9023
:10019E0000B7E075F0DCA4FFAEF0740A8E048F0594
:1001AE00FF12008590079FECF0A3EDF0A208401619
:1001BE0074038C068D07124BB37401124BA5900776
:1001CE009DEEF0A3EFF07E017F00900075E0124BE4
:1001DE00B39000B8E08E048F05FF120085740AFFFD
:1001EE001200858D389000C1E075F0DCA4FFAEF0F2
:1001FE00740A8E048F05FF1200859007A3ECF0A3FE
:10020E00EDF09000C3E060139000C3E0F5F07416BB
:10021E0084FF7E00EF9007ABF0800674649007AB0E
:10022E00F09000A2E0B40B0874E3900064F08049F3
:10023E009000A2E0B419129000B8E0904A1C124B44
:10024E0096E493900064F080309000A2E0B41E1209
:10025E009000B8E0904A3A124B96E493900064F006
:10026E0080179000A2E0B428109000B8E0904A6485
:10027E00124B96E493900064F09000D5E0B4011711
:10028E00900020740FF0A374FFF0900022E4F0A30E
:10029E00F074029000D5F09000D5E0B403419000C8
:1002AE0022E0FEA3E0FF900020E0FCA3E0FD124C54
:1002BE00127410124BB37408124BA5EF900061F03C
:1002CE00EF700674FF900061F074009000D5F0900E
:1002DE000021E0900062F0900020E0900063F0902A
:1002EE000066E090002CF090002CE0241290002D7F
:1002FE00F090002DE0D39424400B90002DE0C39499
:10030E002490002DF0900030E4F090002CE0641169
:10031E00600790002CE0B4122090002CE0B411067F
:10032E007402900030F090002CE0B4120690003071
:10033E007401F0741390002CF090002CE0641460A3
:10034E000790002CE0B4152090002CE0B414067435
:10035E0002900030F090002CE0B41506900030743E
:10036E0001F0741690002CF090002CE064236007CE
:10037E0090002CE0B4242090002CE0B423067402EC
:10038E00900030F090002CE0B42406900030740100
:10039E00F090002C7401F0900031E4F090002DE00C
:1003AE006411600790002DE0B4122090002DE0B48F
:1003BE0011067402900031F090002DE0B4120690F8
:1003CE0000317401F0741390002DF090002DE06454
:1003DE0014600790002DE0B4152090002DE0B414A9
:1003EE00067402900031F090002DE0B415069000D6
:1003FE00317401F0741690002DF090002DE06423FE
:10040E00600790002DE0B4242090002DE0B4230668
:10041E007402900031F090002DE0B424069000316B
:10042E007401F090002D7401F0900066E0FE9000D3
:10043E00C9E02E900033F0900033E0D39424400BAB
:10044E00900033E0C39424900033F0900033E0B476
:10045E0002069000337401F0900033E0B40306748A
:10046E0004900033F0900033E0B412067413900041
:10047E0033F0900033E0B424069000337401F09012
:10048E000033E064126007900033E0B4150690006C
:10049E0033E004F0900033E06411600F900033E01D
:1004AE0064146007900033E0B42306900033E01428
:1004BE00F0900033E0D39412400D900033E0C394DB
:1004CE0012900034F0800A900033E0241290003431
:1004DE00F09000ACE090002EF090002EE0B40206FA
:1004EE0090002E7401F090002EE0B4030674049078
:1004FE00002EF090002EE0B41206741390002EF031
:10050E0090002EE0B41106741090002EF090002E84
:10051E00E0B41406741390002EF090002EE0B41583
:10052E0006741690002EF090002EE0D39412400D1B
:10053E0090002EE0C3941290002FF0800A90002EAF
:10054E00E0241290002FF022C293C294C291C29264
:10055E00C287C290E5B554EFF5B5E5B554DFF5B5F4
:10056E00C296C295C2A0C297C2A2C2A1E5B5547FDF
:10057E00F5B5E5B554BFF5B5E5B554FBF5B5C20D0A
:10058E007536469000AFE0700575480280037548D9
:10059E000390000874FFF0A374DCF0900090E090DC
:1005AE00000EF8E4F0E8A3F0C212C21474C8900072
:1005BE0024F074C8900028F0752500752400C20838
:1005CE00756B00E54AB40903754A00753B0090004F
:1005DE0016E4F0A3F0754B1E752700752600C210A9
:1005EE00C21190079FE0FEA3E0FF7403124BB37499
:1005FE0001124BA590079DEEF0A3EFF0C203900001
:10060E000CE4F0A3F0C21C22053C2285A74E75A770
:10061E00109000ADE0B4031EA2D8B34002C293A264
:10062E00D9B34002C294A2DAB34002C291A2DBB3A4
:10063E004002C2928012A2D8B34004C293C291A2C9
:10064E00D9B34004C294C292A2DCB34002C287A2C4
:10065E00DDB34002C29075D840854EA72290004768
:10066E00E4936406600280FE74C89007A5F8E4F077
:10067E00E8A3F075B50075840175A70075FF807548
:10068E00EF06900032E4F075C91075A70F75A1C77B
:10069E0075A70075D90075CE0C75A70F75F1FE758F
:1006AE00F2FF75F30775F47875A4BA75A5FF75A6F4
:1006BE000775AE0075AFFF75D48175D5FF75D6FF82
:1006CE0075D7FF75A70075A20175A14775F8097555
:1006DE00D80075D90475A71075D80075D90475DAC8
:1006EE000975DB0975DC0975DD0975DE0975DF092C
:1006FE0075D84075A70075E60875E71075BC0175CD
:10070E00BE0475BD6C75BE0775BDA075BE0875BD02
:10071E000175BC0075BB1875BC2075BA0875E880EC
:10072E0075D11375A70F75E10575E20075C740C247
:10073E0093C294C291C292C287C290E5B554EFF5AE
:10074E00B5E5B554DFF5B5C296C295C2A0C297C243
:10075E00A2C2A1E5B5547FF5B5E5B554BFF5B5E533
:10076E00B554FBF5B5759700759780740A12007530
:10077E007597C0E5975420700280F8758F0275A7A3
:10078E0000D2AF75980075A90C75A70F75AB4375A0
:10079E00ADFB75AC1E75A71075C91875CA0075CB63
:1007AE000075C80475A700758912758E04758C00C6
:1007BE00758A00C2A9D28C758D00758B00D2ABD212
:1007CE008E75D944753100753000752D00752C006D
:1007DE00754500754600C2997509C8750800122C3A
:1007EE003975B50074639007A5F8E4F0E8A3F0122C
:1007FE002EC5750964750800122C39C21B90004F66
:10080E00E0B40108A2B54002D21B802E90004FE04A
:10081E00B4021175A70F75F30F75A700A2A34002BE
:10082E00D21B801690004FE0B4030F75A70F75F31F
:10083E001775A700A2A44002D21BA21BB35003023D
:10084E00092F74089007A5F8E4F0E8A3F0122D9490
:10085E00750964750800122C3974099007A5F8E41F
:10086E00F0E8A3F0122D94750964750800122C3966
:10087E00740A9007A5F8E4F0E8A3F0122D94750918
:10088E0064750800122C39740B9007A5F8E4F0E893
:10089E00A3F0122D94750964750800122C39740C8E
:1008AE009007A5F8E4F0E8A3F0122D94750964758D
:1008BE000800122C39740D9007A5F8E4F0E8A3F0A7
:1008CE00122D94750964750800122C39740E900758
:1008DE00A5F8E4F0E8A3F0122D94750964750800EC
:1008EE00122C3974029000AEF090004FE09000721E
:1008FE00F090004FE0B40108740090007AF0801C74
:10090E0090004FE0B4020874009000BDF0800D908E
:10091E00004FE0B4030674009000CAF0D217020A2A
:10092E00089007A5E4F0A304F0122D9475096475E0
:10093E000800122C3974029007A5F8E4F0E8A3F031
:10094E00122D94750964750800122C3974039007E2
:10095E00A5F8E4F0E8A3F0122D947509647508006B
:10096E00122C3974049007A5F8E4F0E8A3F0122DC8
:10097E0094750964750800122C3974059007A5F852
:10098E00E4F0E8A3F0122D94750964750800122C9A
:10099E003974069007A5F8E4F0E8A3F0122D9475CB
:1009AE000964750800122C3974079007A5F8E4F055
:1009BE00E8A3F0122D94750964750800122C397491
:1009CE00019000AEF090004FE0900072F090004F5A
:1009DE00E0B40108740090007AF0801C90004FE0A3
:1009EE00B4020874009000BDF0800D90004FE0B48A
:1009FE00030674009000CAF0C2171230399000B886
:100A0E00E07006740A9000B8F0900064E07006740E
:100A1E00E3900064F0120183E5B54401F5B5740668
:100A2E0090003EF0740190003FF07403900041F08E
:100A3E007404900042F0742D900043F07405900001
:100A4E0044F07403900045F0740090004AF0740076
:100A5E0090004BF0740190004CF0740090004DF03B
:100A6E0074FF90004EF0745390013CF07475900139
:100A7E003DF0746290013EF0746190013FF074722B
:100A8E00900140F07475900141F07420900142F095
:100A9E007434900143F07443900144F074799001E2
:100AAE0045F0746C900146F07420900147F0743359
:100ABE00900148F07436900149F0745490014AF058
:100ACE009000D4E0900061F090008BE0900062F016
:100ADE0090008CE0900063F0C212C21474C89000B3
:100AEE0024F074C8900028F0C210C211A2B6B392BE
:100AFE0009A2B3B3920A75250075240075364675A2
:100B0E004B1E90005DE4F075261975276490000861
:100B1E0074FFF0A374DCF0C20D754A00C20875298B
:100B2E000075280090000CE4F0A3F0743A9007656D
:100B3E00F074FD900766F0756C0090005EE4F07541
:100B4E002B00752A00900010E4F0A3F0900090E0C6
:100B5E0090000EF8E4F0E8A3F0900071E075F0322A
:100B6E00A4FFAEF090001EEEF0A3EFF090079FE012
:100B7E00FEA3E0FF7403124BB37401124BA5900752
:100B8E009DEEF0A3EFF075490174FA90003AF0C2B1
:100B9E001C756B00753B00C20EC20FC21DC20375E1
:100BAE004C00C204D205C206D207C218C219D21A0C
:100BBE0074FE900035F074FE900036F075370075B7
:100BCE004300753900753D32753E00753F00743C2B
:100BDE00900038F0754000743C900039F07541007B
:100BEE00754200900016E4F0A3F0754400D2B2D224
:100BFE00A4D2B0D2B1D2A3D2A7D2A6D2A5D2B79048
:100C0E000071E0D394FA400674FA900071F07E0100
:100C1E007F00900063E0124BB3900062E02FFF5014
:100C2E00010E900020EEF0A3EFF0EFD394FFEE94C0
:100C3E000F4007900020E4F0A3F0900061E07006F2
:100C4E0074FF900061F09000AEE0D3940240067401
:100C5E00019000AEF09000AFE07005754802800381
:100C6E007548039000B0E0D39401400674009000E4
:100C7E00B0F09000B6E0C3940A5006740A9000B625
:100C8E00F09000C0E0700674019000C0F09000C0BB
:100C9E00E0B4FF0674FE9000C0F09000C7E0D3945D
:100CAE00FE400674FE9000C7F074019000CDF07403
:100CBE00019000CEF074009000D0F074009000D53A
:100CCE00F0D29CD2EC75CF01A298B350030210C3A0
:100CDE00C298E54664046006E59964FF6002801ED2
:100CEE00E546600874E6254690003AF0754600E544
:100CFE0045600874F0254590003AF0754500E546CC
:100D0E006003020DAE754600E599B4FF037545010B
:100D1E00E599B4FE03754502E599B4FD03754503E7
:100D2E00E599B4FC03754504E599B4FA03754505D8
:100D3E00E599B4FB03754601E599B4F903754604CC
:100D4E00E599D394E54007E599C394F040028016E7
:100D5E008599477546027E017F00E547C394E612EA
:100D6E004BB38E2E8F2F753100753000E599D394CD
:100D7E00C74007E599C394E64002801F85994775E1
:100D8E00460374E5C39547F52F752E00AE2EAF2F93
:100D9E009047E31200647830124BF8D2990210C3D8
:100DAE00E546B401028003020E8AE5314530700338
:100DBE00120556AE30AF31900065124BDAE599F060
:100DCE007830124C1AAE30AF31EFB40106EEB407E4
:100DDE00028003020E8A900765E0B43C0280030293
:100DEE000E74C29C120183900061E09000D4F090CA
:100DFE000062E090008BF0900063E090008CF0A217
:100E0E00174031754F01E54FD394075025E54F90AC
:100E1E0007A5F8E4F0E8A3F074AA900032F0122CC3
:100E2E0065750964750800122C39784F740126F621
:100E3E0050D4802F754F08E54FD3940E5025E54FB3
:100E4E009007A5F8E4F0E8A3F074AA900032F0122F
:100E5E002C65750964750800122C39784F740126BB
:100E6E00F650D412303974C89007A5F8E4F0E8A310
:100E7E00F0D29C7546007545007599FBE546B402A7
:100E8E00028003020F1EE5314530700685992D75DF
:100E9E002C00AE30AF3174016F4E701BAC2CAD2DEB
:100EAE00AA2EAB2FED2BFBEC3AFA8A068B0790009D
:100EBE0065124BDAE599F07830124C1AAE30AF313C
:100ECE0074026F4E704AAC2CAD2D740D6D4C7027A4
:100EDE0074639007A5F8E4F0E8A3F074AB900032C9
:100EEE00F0900072E090004FF0122F9E74C89007A1
:100EFE00A5F8E4F0E8A3F0AE2CAF2D74566F4E704B
:100F0E0003120556120183854799754600754500F3
:100F1E00E546B4033FAE30AF31900065124BDAE5D3
:100F2E0099F07830124C1AAE30AF31AC2EAD2F8F07
:100F3E00028E038C068D0790481F120064E493F90D
:100F4E00740193FEEAD39EEB994009854799754645
:100F5E0000754500E546B4040280030210C3E53176
:100F6E0045307003120556AE30AF31900065124B0E
:100F7E00DAE599F07830124C1AAE30AF31EFB4009A
:100F8E0006EEB4010280030210C3900048E075F033
:100F9E0002A4FDACF08D4FED900065124BEFEDFA13
:100FAE00E0FBEA900068124BEFEBFAE0FBEA2BFA5B
:100FBE00900048E0B5020280030210B50DED9000DE
:100FCE0065124BEFE54FFDE0FAED900069124BEF25
:100FDE00EAFDE0FAEDC39AFD900048E0B505028007
:100FEE00030210B5E54F900067124BEFE54FFDE0A1
:100FFE00FAED90006A124BEFEAFDE0FAED2AFD9051
:10100E000048E0B5050280030210B5E54F90006B75
:10101E00124BEFFDE0FAED900048E0F4042A900048
:10102E004FF0E54F90006C124BEFFDE0FAED9000A3
:10103E0048E0F4042A900050F0E54F90006D124BFA
:10104E00EFFDE0FAED900048E0F4042A900051F034
:10105E00E54F90006E124BEFFDE0FAED900048E088
:10106E00F4042A9007A5F8E4F0E8A3F074AB90001E
:10107E0032F0122F9E750964750800122C399007F4
:10108E00A5124BC1122F9E750964750800122C39DA
:10109E009007A5124BC1122F9E7599F975096475AB
:1010AE000800122C3980FE7599FF750964750800C9
:1010BE00122C3980FEE5456006A299B3B3400302B7
:1010CE001224C299E545B4011FAE30AF3190003EF7
:1010DE00124BDAE0F5997830124C1AAE30AF31740B
:1010EE00116F4E7003754500E545B40203854999AD
:1010FE00E545B4031DAE30AF31900065124BDAE01A
:10110E00F599EFB40107EEB4070375450078301278
:10111E004C1AE545B404028003021203E531453052
:10112E007003852599AE30AF3174016F4E70038513
:10113E003799AE30AF3174026F4E7003853999AE68
:10114E0030AF3174036F4E7003853D99AE30AF31C1
:10115E0074046F4E7003853F99AE30AF3174056FD6
:10116E004E7003854099AE30AF3174066F4E7003EA
:10117E00854199AE30AF3174076F4E700385429939
:10118E00AE30AF3174086F4E7006900017E0F599CF
:10119E00AE30AF3174096F4E700690003AE0F5999B
:1011AE00AE30AF31740A6F4E7003854399AE30AFD7
:1011BE0031740B6F4E7003853E99AE30AF31740CA7
:1011CE006F4E7003854499AE30AF31740D6F4E7013
:1011DE000590003AE4F0AE30AF31740D6F4E7003EF
:1011EE007599FC7830124C1AAE30AF31740E6F4ECA
:1011FE007003754500E545B4051CAE30AF3190491E
:10120E004D124BDAE493F59974E36F4E7003754506
:10121E00007830124C1AE54664016005E546B404C8
:10122E0003020CD3C28E7E107F00E53C124BB3E559
:10123E008D75F010A4FDACF0EF2DFDEE3CFCE58BB2
:10124E0075F01084FF7E00ED2FFFEC3EFE8E268F94
:10125E0027D28E900092E06056900018124BC190EB
:10126E000018E0FCA3E0FD90001AE0FAA3E0FBED0D
:10127E00B5033CECB50238B216A208B34013A21661
:10128E00B34008E5B54404F5B58006E5B554FBF565
:10129E00B590001AE0FEA3E0FF90001CE0FCA3E076
:1012AE00FDEF2DFDEE3CFC90001AECF0A3EDF0905E
:1012BE00009FE0600990009FE0C394034002806F9E
:1012CE00124539A208B3500990005DE0C394464020
:1012DE00028006900089E0F56AE56A75F005A4FFC4
:1012EE00AEF09007A7EEF0A3EFF0900076E0C39576
:1012FE00394007E537C3953850079007A7E4F0A3A8
:10130E00F0AE57AF589007A7E0FCA3E0FDEFD39DDA
:10131E00EE9C4004C2A1800B90005DE0C39464502B
:10132E0002D2A190009FE0B40205A2A1B392A290B6
:10133E00009FE0B4031C124635AE57AF589007A776
:10134E00E0FCA3E0FDEFD39DEE9C4004D2A1800211
:10135E00C2A190007AE06009A2B3300A01B3B34093
:10136E00028039A2B3300A01B34031A2B3300C016E
:10137E00B3401C9000ADE0B40306A218B3B3400214
:10138E008006740590003AF0D218A20CB3920AA20D
:10139E000CB330B301B34004A20C920AA2B63009CA
:1013AE0001B35003021907A2B6300901B35003026C
:1013BE001907A2B6300B01B350030218217549006C
:1013CE00900092E07013A20BB34008E5B554FBF504
:1013DE00B58006E5B54404F5B50536A20DB3B35098
:1013EE0013AE26AF27900008E0FCA3E0FDEDC39FEF
:1013FE00EC9E40030214EFE536B411067536130267
:10140E0014D2E548B40330E536B42305754801809F
:10141E001FA21CB3401AE536C39423500690003A1F
:10142E007401F0E536D394234006740290003AF02E
:10143E00753601D21C8044E548B402067548017524
:10144E003623E536B42305753601802F90003AE039
:10145E00701AE536C39423500690003A7401F0E5F5
:10146E0036D394234006740290003AF09000AFE019
:10147E00B402051205568003753601900092E060A5
:10148E0043900018E0FEA3E0FF900092E08E048FE0
:10149E0005FF12008574018C068D07124BA5900076
:1014AE001CEEF0A3EFF090001CE0F8A3E090001A01
:1014BE00C8F0A3C8F0900018E4F0A3F0C216E5B58A
:1014CE0054FBF5B5AE28AF29AC26AD27EF2DFDEEBA
:1014DE003CFC74028C068D07124BA58E288F29803A
:1014EE002BAE28AF29AC26AD27EF2DFDEE3CFC74BC
:1014FE00018C068D07124BA58E288F29AC26AD27A1
:10150E00EDD39410EC94274003120556E536B4142F
:10151E0003753616E536B42310740390003AF09036
:10152E0000AFE0B40203120556AE2AAF2BAC26ADC7
:10153E0027EF2DFDEE3CFC8C2A8D2BAE26AF27EF30
:10154E00D39DEE9C4011900010E0FAA3E0FBEBC39C
:10155E0094E8EA940340028006900010124BC1906A
:10156E00000CE0FEA3E0FFAC26AD27EF2DFDEE3C18
:10157E00FC90000CECF0A3EDF09000AFE0B402187C
:10158E00AE26AF277405124BB37401124BA5900013
:10159E0008EEF0A3EFF08011AE26AF277402124BC7
:1015AE00B3900008EEF0A3EFF0C28E758D00758B30
:1015BE0000753C00752701752600D28EE53624088D
:1015CE0075F00984AFF07E00EF4E707590000CE060
:1015DE00F8A3E090000AC8F0A3C8F090000AE0FE5D
:1015EE00A3E0FFEF4E600B7C7B7D89124AB58E2403
:1015FE008F2590000CE4F0A3F0AE24AF257428BE26
:10160E0000039F5010E53B2FFF50010E7401124B4B
:10161E00A58E248F2585253B9000B6E0A824B80022
:10162E000DD395254008E525900037F080099000F0
:10163E00B6E014900037F0E5486006752500752475
:10164E00009000ADE0B4030890002EE06536600215
:10165E008026A218B34004D2198002B21990007AE3
:10166E00E0600BA218B35006A219B3B34002800675
:10167E00740490003AF0C218E536640B6005E53646
:10168E00B41D0990009FE0600312427B900033E08E
:10169E0065366007900034E0B53603754A00A20E39
:1016AE00500302178990006BE0B4015AE53F75F0C4
:1016BE000584FF7E00900565124BDAE0F533753236
:1016CE0000AE32AF33900069E0124BB374648E04F7
:1016DE008F05FF12008574C18C068D07124BB38ED9
:1016EE00348F3590000EE0FEA3E0FFAC32AD331226
:1016FE00000374648E048F05FF12008590000EECBB
:10170E00F0A3EDF0800F900069E075F0C1A4FFAE7C
:10171E00F08E348F35E539C394CC505D75A71085A6
:10172E00F94F85FA507E017F00E550124BB3E54F1D
:10173E002FFF50010E8E328F33AC34AD35EF2DFDB1
:10174E00EE3CFC8C348D35D293D294E535F5FBE529
:10175E0034F5FCE535F5E9E534F5EA9000ADE0B495
:10176E000314D291D292E535F5EBE534F5ECE5357F
:10177E00F5EDE534F5EE75A700D20EE548B4010699
:10178E00E536640B6002800F754B0190003D7401CD
:10179E00F0E5B54401F5B5E54870739000B2E06030
:1017AE000D9000B9E0A824B80006952540028032BD
:1017BE009000B2E0B4021790002CE06536600790FE
:1017CE00002DE0B53603754B03754400800CC20046
:1017DE00754400900016E4F0A3F0740990003AF0FE
:1017EE00802C90002CE06536600790002DE0B53619
:1017FE0003754B0190002CE0B5360690003D740148
:10180E00F090002DE0B53606740290003DF0A20B6C
:10181E00B39209A20BB330B601B350030219077588
:10182E004901900092E07013A20BB34008E5B54455
:10183E0004F5B58006E5B554FBF5B5A20B9209E5A6
:10184E0036D3944A4012D20DE536D39468400974CB
:10185E000390003AF07536469000BAE0B40107E501
:10186E0042C3941440028003120556744690005DE4
:10187E00F0A204300501B35017A204B34008E5B539
:10188E004408F5B58006E5B554F7F5B5A204920502
:10189E00A206300701B35017A206B34008E5B544BF
:1018AE0002F5B58006E5B554FDF5B5A2069207E53D
:1018BE0042C394415009740E90003AF012055690AE
:1018CE000044E0FE900040E0C39E4009900040E0DE
:1018DE00D39406400974FB90003AF012055690001E
:1018EE0049E06015900049E0FE900043E06E60090B
:1018FE0074FE90003AF0120556A210B3B350089041
:10190E00002EE0653660030219E5A202B35006A26E
:10191E0000B3B340030219E175A71085F94F85FA9C
:10192E00507E017F00E550124BB3E54F2FFF500163
:10193E000E8E328F33900014E0FCA3E0FDEF2DFDF0
:10194E00EE3CFC8C348D359000ADE0B4034EA20815
:10195E00B34028A219B3400CE535F5FBE534F5FC90
:10196E00D293800AE535F5EBE534F5ECD291A2037E
:10197E00B34004D2A08002C2A0801FE535F5FBE57E
:10198E0034F5FCE535F5EBE534F5ECD293D291A2C6
:10199E0003B34004D2A08002C2A08011E535F5FB4E
:1019AE00E534F5FCD293A203B34002D2919000CB62
:1019BE00E0B4021CAE32AF33AC55AD56EF2DFDEE9A
:1019CE003CFC8C348D35E535F5FDE534F5FED287DE
:1019DE0075A700C210D211A211B3B3500890002FF8
:1019EE00E065366003021AC3A202B35006A200B32A
:1019FE00B34003021ABF75A71085F94F85FA507EC2
:101A0E00017F00E550124BB3E54F2FFF50010E8EB4
:101A1E00328F33900014E0FCA3E0FDEF2DFDEE3C81
:101A2E00FC8C348D359000ADE0B4034EA208B3406B
:101A3E0028A219B3400CE535F5E9E534F5EAD29460
:101A4E00800AE535F5EDE534F5EED292A203B3400A
:101A5E0004D2A08002C2A0801FE535F5E9E534F579
:101A6E00EAE535F5EDE534F5EED294D292A203B364
:101A7E004004D2A08002C2A08011E535F5E9E5341C
:101A8E00F5EAD294A203B34002D2929000CBE0B416
:101A9E00021CAE32AF33AC55AD56EF2DFDEE3CFC15
:101AAE008C348D35E535F5CEE534F5CFD29075A76E
:101ABE0000D210C211E54BB40816123BAAA210B305
:101ACE005005A211B340028004D210D211754B1EE4
:101ADE00E54BB40706123962754B08E54BB4063D6B
:101AEE0090000EE0FEA3E0FFEF4E6006A208B3B337
:101AFE0040028023AE51AF5290000EE0FCA3E0FDF9
:101B0E00EF2DFDEE3CFC8C518D52E536D3941250E8
:101B1E000690000E120039123734754B07E54BB4A0
:101B2E000506123594754B06E54BB404329000A0B1
:101B3E00E0902C1BF82828731232288012123228BB
:0F1B4E00800D1233D68008123488800312348839
:0F2C1B00021B46021B4B021B50021B55021B5A89
:101B5D00900082E060051243648002C204754B055B
:101B6D00E54BB403028003021C57900085E060052D
:101B7D001244548002C2069000A0E0D39402403F6C
:101B8D00900074E02403A824B80004952550099012
:101B9D000076E0D3953950028008D2027408900087
:101BAD003AF0900074E0A824B80005D39525500BA9
:101BBD00900076E02403C395395002C2028039901B
:101BCD000074E02403A824B8000495255007E537D8
:101BDD00C3953840028008D202740890003AF09004
:101BED000074E0A824B80005D395255009E53824E4
:101BFD000FC395375002C2029000BAE07007E5425C
:101C0D00C3941440028002D202A2024005754B0417
:101C1D00800A754B1E900016E4F0A3F0A208B340A5
:101C2D0029E53F75F00584FF7E00900565124BDABE
:101C3D00E0C3946950051242B0800F90079FE0F801
:101C4D00A3E090079DC8F0A3C8F0E54BB40A02804D
:101C5D0003021D19900026E0C394465008C29674E5
:101C6D0046900026F0900030E0B4011DE559240A9D
:101C7D00F5599007A1E0FEA3E0FF740A2FFF500174
:101C8D000E9007A1EEF0A3EFF0900030E0B4021D2E
:101C9D00E5592414F5599007A1E0FEA3E0FF741453
:101CAD002FFF50010E9007A1EEF0A3EFF0855933F1
:101CBD0075320090002CE0F54F12009EE535900036
:101CCD0026F0900004E532F0A3E533F0E54F9000E7
:101CDD0027F0C2139007A1E0F532A3E0F533900091
:101CED002CE0F54F12009EE535900024F090000099
:101CFD00E532F0A3E533F0E54F900025F0C212E593
:101D0D0048B40105754B0B8003754B03900024E01F
:101D1D00B536028003021DB8A2124072900000E099
:101D2D00FEA3E0FFEF4E6021AE28AF29900000E04A
:101D3D00FCA3E0FD120003740A8E048F05FF120050
:101D4D0085900000ECF0A3EDF0900025E0601A9076
:101D5D000000E0FEA3E0FFAC28AD29EF2DFDEE3C29
:101D6D00FC900000ECF0A3EDF0900025E0D3940181
:101D7D00401A900000E0FEA3E0FFAC28AD29EF2D46
:101D8D00FDEE3CFC900000ECF0A3EDF0D212AE267F
:101D9D00AF27900000E0FCA3E0FDEFC39DEE9C405B
:101DAD000AD296C21274C8900024F0A212B3B35096
:101DBD0007900024E0B53602800AD29674C89000D0
:101DCD0024F0C212900026E0B536028003021E7088
:101DDD00A2134072900004E0FEA3E0FFEF4E6021DD
:101DED00AE28AF29900004E0FCA3E0FD12000374BF
:101DFD000A8E048F05FF120085900004ECF0A3ED10
:101E0D00F0900027E0601A900004E0FEA3E0FFAC24
:101E1D0028AD29EF2DFDEE3CFC900004ECF0A3ED78
:101E2D00F0900027E0D39401401A900004E0FEA347
:101E3D00E0FFAC28AD29EF2DFDEE3CFC900004EC4D
:101E4D00F0A3EDF0D213AE26AF27900004E0FCA373
:101E5D00E0FDEFC39DEE9C400AC2967446900026AD
:101E6D00F0C213A213B3B35007900026E0B53602AB
:101E7D00800AC2967446900026F0C213E54BB40B4F
:101E8D00028003021F5590002AE0C394465008C2F9
:101E9D0095744690002AF0900031E0B4011DE5598B
:101EAD00240AF5599007A1E0FEA3E0FF740A2FFF65
:101EBD0050010E9007A1EEF0A3EFF0900031E0B4C9
:101ECD00021DE5592414F5599007A1E0FEA3E0FF8A
:101EDD0074142FFF50010E9007A1EEF0A3EFF085C3
:101EED00593375320090002DE0F54F12009EE53507
:101EFD0090002AF0900006E532F0A3E533F0E54FAF
:101F0D0090002BF0C2159007A1E0F532A3E0F53358
:101F1D0090002DE0F54F12009EE535900028F090D1
:101F2D000002E532F0A3E533F0E54F900029F0C251
:101F3D0014E548B4010F75480074C8900024F0747E
:101F4D00C8900028F0754B03900028E0B53602804C
:101F5D0003021FF4A2144072900002E0FEA3E0FF02
:101F6D00EF4E6021AE28AF29900002E0FCA3E0FD0A
:101F7D00120003740A8E048F05FF12008590000273
:101F8D00ECF0A3EDF0900029E0601A900002E0FE65
:101F9D00A3E0FFAC28AD29EF2DFDEE3CFC90000237
:101FAD00ECF0A3EDF0900029E0D39401401A9000DD
:101FBD0002E0FEA3E0FFAC28AD29EF2DFDEE3CFCC9
:101FCD00900002ECF0A3EDF0D214AE26AF279000F6
:101FDD0002E0FCA3E0FDEFC39DEE9C400AD295C24A
:101FED001474C8900028F0A214B3B35007900028C1
:101FFD00E0B53602800AD29574C8900028F0C2145C
:10200D0090002AE0B5360280030220ACA215407282
:10201D00900006E0FEA3E0FFEF4E6021AE28AF2951
:10202D00900006E0FCA3E0FD120003740A8E048FFD
:10203D0005FF120085900006ECF0A3EDF090002B4B
:10204D00E0601A900006E0FEA3E0FFAC28AD29EF9A
:10205D002DFDEE3CFC900006ECF0A3EDF090002B76
:10206D00E0D39401401A900006E0FEA3E0FFAC28F7
:10207D00AD29EF2DFDEE3CFC900006ECF0A3EDF04C
:10208D00D215AE26AF27900006E0FCA3E0FDEFC30E
:10209D009DEE9C400AC295744690002AF0C215A28E
:1020AD0015B3B3500790002AE0B53602800AC295E9
:1020BD00744690002AF0C215E54BB4027612401317
:1020CD0012412A90079DE0FEA3E0FF740A124BB364
:1020DD0090000AE0FCA3E0FD74098F02FF12008559
:1020ED008D078C038E048A058B06124AB59007A1C5
:1020FD00EEF0A3EFF074F0BE00039F500B74F09060
:10210D0007A1F8E4F0E8A3F09007A1E0FEA3E0FF3B
:10211D00E5592FFF50010E9007A1EEF0A3EFF090BF
:10212D00003DE0B40103754B0A90003DE0B402039D
:10213D00754B0BE54BB401259000D2E0902C2AF89D
:10214D00282873123DB18012123DB1800D123E3B15
:0A215D008008123EE78003123EE7FF
:0F2C2A0002215002215502215A02215F0221642A
:10216700754B029000BDE0B4020280030222829008
:102177000060E0D3953E5064900060E0F404253E93
:10218700FE9000C0E08E00F5F0E884FF7E008F4FE0
:10219700EFC39410500CEF854FF0A4FDACF08D4FBA
:1021A7008003754FFF900060E0D3954F400B900080
:1021B70060E0C3954FF54C8003754C009000DBE061
:1021C700D3954C40069000DBE0F54C9000DCE0C373
:1021D700954C50069000DCE0F54C8071900060E073
:1021E700C3953EFE9000C0E08E00F5F0E884FF7EC8
:1021F700008F4FEFC39410500CEF854FF0A4FDAC48
:10220700F08D4F8003754FFF854F33753200900077
:1022170060E02533FFAE3250010E8E328F3374FFEC
:10222700BE0009D39F400585334C8003754CFF9052
:1022370000DBE0D3954C40069000DBE0F54C9000C6
:10224700DCE0C3954C50069000DCE0F54CA208B3E7
:10225700B350099000C8E0D3954D5002800A740727
:1022670090003AF0C297801375A710E5CDC3954C3F
:102277004004C2978002D29775A700E54AC3940924
:1022870040030229BDA2EDB350030229BDC2EDE50B
:102297004A600302243190006EE07003022420900C
:1022A70000A4E0B401028003022380900033E0B56C
:1022B7003602800302237D7E017F00E5BE124BB309
:1022C700E5BD2FFF50010E8E328F3390006EE0B4C4
:1022D70001187410124BB3900064E08E048F05FF51
:1022E700120085ED900035F0802CAE32AF337410BC
:1022F700124BB3900064E08E048F05FF12008590A7
:102307000035E02DFD50010C74018C068D07124B32
:10231700A5EF900035F0E54360089000CAE064023D
:10232700600280219000CCE0B4011A900035E0757E
:10233700F0E7A4FFAEF0E5438E048F05FF1200859A
:10234700ED900035F0900035E0FE900036E0D39E2A
:102357004004D21A8002B21A900035E0900036F09D
:102367009000A0E064016006A21AB3B340028006A1
:10237700900035E0F53702241ED21A7E017F00E572
:10238700BE124BB3E5BD2FFF50010E8E328F339037
:10239700006EE0B401187410124BB3900064E08E25
:1023A700048F05FF120085ED900035F0802CAE32CA
:1023B700AF337410124BB3900064E08E048F05FFA7
:1023C700120085900035E02DFD50010C74018C063C
:1023D7008D07124BA5EF900035F0E543600890009C
:1023E700CAE06402600280219000CCE0B4011A9038
:1023F7000035E075F0E7A4FFAEF0E5438E048F05E6
:10240700FF120085ED900035F09000A0E0640160B8
:1024170006900035E0F537800375370090006AE0D5
:102427007005754A01800375BB18E54AB40102803F
:10243700030225D390006AE070030225C27E017F64
:1024470000E5BE124BB3E5BD2FFF50010E8E328F54
:10245700339000B0E0B4010F7E0F7FFFAC32AD3395
:10246700124C128E328F339000D5E0B40245AE3253
:10247700AF33900020E0FCA3E0FDEDD39FEC9E403E
:102487000A900020E532F0A3E533F0AE32AF339087
:102497000022E0FCA3E0FDEFD39DEE9C400A9000F4
:1024A70022E532F0A3E533F0AE32AF337404124BBA
:1024B700A58F399000D5E0704CAE32AF3390002035
:1024C700E0FCA3E0FDEFD39DEE9C4009124C128E79
:1024D700328F338006753300753200AE32AF3374F6
:1024E70010124BB3900061E08E048F05FF12008538
:1024F7008C328D337400D39D74019C40058533392C
:1025070080037539FF9000A0E0B401028003022523
:10251700C0A208B3B3500E900074E0A824B8000519
:10252700D3952550030225B5900075E075F019A4E1
:10253700FFAEF09000B8E08E048F05FF1200859083
:1025470000B1E08539F0A4FFAEF074648D028C030E
:102557008E048F05FF120085EA2DFDEB3CFC8C32C3
:102567008D33E543600F9000CAE0B402089000CCB9
:10257700E0640160028017AE32AF3374E7124BB3E9
:10258700E5438E048F05FF1200858C328D33900052
:1025970035E0A832B8000AD3953340058533378034
:1025A7000BA21AB34006900035E0F537800BA21A4C
:1025B700B34006900035E0F5378003753900900089
:1025C7006DE07005754A02800375BB19E54AB402D0
:1025D70002800302268E90006DE0700302267DE5DF
:1025E70036D39412400302267B90001EE0FEA3E040
:1025F700FFE53D124C0A90001EEEF0A3EFF07E01BE
:102607007F00E5BE124BB3E5BD2FFF50010E8E32A2
:102617008F339000DAE07013740A124BB374518E43
:10262700048F05FF1200858D3D8019AE32AF3374DC
:102637000A124BB38F048E057E017F95CDCCCD1248
:102647004AB58F3DE53DD394644003753D649000E2
:102657001EE0FEA3E0FFE53D2FFF50010E90001E98
:10266700EEF0A3EFF0900071E0048E048F05FF12E7
:1026770000858D3D8003753D329000BDE070057586
:102687004A03800375BB13E54AB4035E9000BDE0BF
:1026970060477E017F00E5BE124BB3E5BD2FFF50BB
:1026A700010E8E328F337404124BA58F3E9000BFFC
:1026B700E0853EF0A4FDACF07464FF1200858D3E0A
:1026C7009000BEE0853EF0A4FFAEF074FF8E048F4D
:1026D70005FF1200858D4D8003753E0090006BE06D
:1026E7007005754A04800375BB17E54AB404028078
:1026F7000302278F90006BE0B4017C7E017F00E529
:10270700BE124BB3E5BD2FFF50010E7404124BA54B
:102717008E328F33900038E06012900038E01490CA
:10272700485B93A832B800069533400280069000B4
:1027370038E014F0900038E0C394775013900038D5
:10274700E00490485B93A832B80005D39533500254
:102757008006900038E004F0900038E0FE90009189
:10276700E08E0088F0A4FFAEF074648E048F05FF3E
:102777001200858D3F8003753F0090006CE0700567
:10278700754A05800375BB16E54AB4050280030246
:10279700282290006CE0B4017C7E017F00E5BE1228
:1027A7004BB3E5BD2FFF50010E7404124BA58E32BB
:1027B7008F33900039E06012900039E0149048D4CC
:1027C70093A832B80006953340028006900039E09E
:1027D70014F0900039E0C394775013900039E00467
:1027E7009048D493A832B80005D395335002800699
:1027F700900039E004F0900039E0FE900097E08EF9
:102807000088F0A4FFAEF074648E048F05FF1200F9
:10281700858D40800375400075BB1FE54AB40633BC
:102827007E017F00E5BE124BB3E5BD2FFF50010EC1
:102837008E328F337409124BB374E68E048F05FF03
:102847001200858D42900073E07005754A0780037A
:1028570075BB15E54AB4070280030229649000732B
:10286700E070030229537E017F00E5BE124BB3E5FA
:10287700BD2FFF50010E8E328F337404124BA58F7C
:1028870041900073E0B401159000C7E08541F0A4C2
:10289700FFAEF07407124BA5EF9007AAF0900073F4
:1028A700E0B402159000C7E08541F0A4FFAEF074D4
:1028B70007124BA5EF9007A9F0900073E0B403024D
:1028C70080030229519000B4E0701CE541C3940ACB
:1028D7005002D201E541D394644002C201900093B3
:1028E700E090005FF08063900093E070349000C741
:1028F700E08541F0A4FFAEF074FF8E048F05FF1250
:102907000085ED90005FF0AE24AF25741EBE000673
:10291700D39F4002D201E539D394E54002C201803A
:1029270029E541C3940A500DAE24AF25741EBE009D
:1029370004D39F50028002D201E539D394E54002C7
:10294700C201900093E090005FF080037541009012
:1029570000CAE07005754A08800375BB14E54AB4E0
:1029670008509000CAE060397E017F00E5BE124B37
:10297700B3E5BD2FFF50010E8E328F33EFD3942175
:10298700EE940E40057543FF8015AE32AF337410D9
:10299700124BB374E38E048F05FF1200858D4380BD
:1029A7000375430090006EE0600575BB1A800375E0
:1029B700BB18054AD2ECAE26AF27EFD39410EE949E
:1029C700275003022C18C20D7536469000AFE070F1
:1029D700057548028003754803C293C294C291C229
:1029E70092C287C290E5B554EFF5B5E5B554DFF56A
:1029F700B5C296C295C2A0C297C2A2C2A1E5B554FC
:102A07007FF5B5E5B554BFF5B5A21BB34008E5B5ED
:102A17004404F5B58006E5B554FBF5B5A20FB350F0
:102A27000EE539D394334007E539C394CC4003020C
:102A37002AC2E5B54401F5B5744690005DF09000F3
:102A470069E075F064A4FFAEF08E348F357402BE72
:102A5700000AD39F400675350275340075A71085A7
:102A6700F94F85FA507E017F00E550124BB3E54FD1
:102A77002FFF50010E8E328F33AC34AD35EF2DFD65
:102A8700EE3CFC8C348D35D293D294E535F5FBE5DD
:102A970034F5FCE535F5E9E534F5EA9000ADE0B449
:102AA7000314D291D292E535F5EBE534F5ECE53533
:102AB700F5EDE534F5EE75A700D20FE539C3941AA5
:102AC7005002C20F90000874FFF0A374DCF090006E
:102AD70090E090000EF8E4F0E8A3F0C212C214747C
:102AE700C8900024F074C8900028F0C210C2117575
:102AF7002500752400753B00C208756B0090001611
:102B0700E4F0A3F0754B1E90079FE0FEA3E0FF746F
:102B170003124BB37401124BA590079DEEF0A3EF80
:102B2700F0900082E060051243648002C2049000C6
:102B370085E060051244548002C206A204300501F4
:102B4700B35017A204B34008E5B54408F5B58006AD
:102B5700E5B554F7F5B5A2049205A206300701B30F
:102B67005017A206B34008E5B54402F5B58006E55F
:102B7700B554FDF5B5A2069207C203752B00752A59
:102B870000900010E4F0A3F0900071E075F032A41B
:102B9700FFAEF090001EEEF0A3EFF090000CE4F013
:102BA700A3F0C21C90005EE0C3943C5019758D6E73
:102BB700758B00753C02E54AB4090990005EE00494
:102BC700F0754A00803BE54AB40903754A0075274A
:102BD70000752600758D00758B00753C0090005DB3
:102BE700E0C39464500890005DE004F080067464CC
:102BF70090005DF090005DE0B46406E5B554FEF525
:102C0700B5E542C394415009740E90003AF012059D
:042C170056020CD382
:1047E3000000010001400160018001A001C001E05F
:1047F30002000300039603B603D603F40400050086
:1048030005180530054805600578059005A805C01D
:10481300060006140628063C066E068C00FF013FC0
:10482300015F017F019F01BF01DF01FF02FF0395CC
:1048330003B503D503F303FF04FF0517052F05474E
:10484300055F0577058F05A705BF05FF0613062737
:10485300063B066F068B06A9DAD8D7D5D4D2D0CFBC
:10486300CDCBC9C7C6C4C2C0BEBCBAB8B5B3B1AF5D
:10487300ADABA8A6A4A2A09D9B99969492908D8B74
:1048830089878482807E7C79777573716F6D6B699C
:10489300676563615F5D5B5957565452504F4D4B8B
:1048A3004A4847454442413F3E3C3B3A3937363517
:1048B300343231302F2E2D2C2B2A2928272625253B
:1048C3002423222121201F1E1E1D1C1C1B1A1A1902
:1048D30019EEECEBEAE9E8E7E5E4E3E1E0DEDDDB52
:1048E300D9D8D6D4D2D0CECCCAC8C6C3C1BFBCBA1D
:1048F300B7B5B2B0ADABA8A5A3A09D9B9895929078
:104903008D8A8785827F7D7A7775726F6D6A686518
:1049130063615E5C5A575553514F4D4B494745436D
:1049230042403E3C3B393836353332312F2E2D2B26
:104933002A292827262524232221201F1E1D1D1C4A
:0A4943001B1A1A191818171616157A
:102C3900750B00750A00AE0AAF0BAC08AD09EDC300
:102C49009FEC9E401674FF12007575CF01780B74C6
:102C59000126F6500418E436F650DB22900032E0E3
:102C6900B4AA1C900765E0B43C159007A5E0FEA343
:102C7900E0FFEF4E6009741EBE0004D39F500302AB
:102C89002D9375350075340075F8099007A5E0FE98
:102C9900A3E0FF74076F4E6006740E6F4E700674E2
:102CA9003A900765F09007A5E0FEA3E0FF7408BE1F
:102CB900001ED39F401A7E017F089007A5E0FCA360
:102CC900E0FD1DBDFF011C1200038E328F33801FF2
:102CD9009007A5E0FEA3E0FF7408124C0A8F048E4A
:102CE900057E017F08CDCCCD1200038E328F33AE25
:102CF90034AF35740CD39F74019E5003022D8EA2FC
:102D0900F9B3407EE5354534700375A382AE34AF1F
:102D19003574016F4E700375A300AE34AF3574027C
:102D29006F4E700D9007A6E075F002A4FDACF08D12
:102D3900A3AE34AF3574036F4E700375A300AE3480
:102D4900AF357403BE00039F5013AC32AD33ED2F82
:102D5900FFEC3EFE900061124BDAE0F5A3AE34AF12
:102D690035EFB40B09EEB401057414120075AE34D5
:102D7900AF35EFB40B07EEB4010375F80D783412D3
:102D89004C1A022CF8900032E4F0227535007534A3
:102D99000075F8099007A5E0FEA3E0FF7408BE00DE
:102DA9001ED39F401A7E017F089007A5E0FCA3E08F
:102DB900FD1DBDFF011C1200038E328F33801F9051
:102DC90007A5E0FEA3E0FF7408124C0A8F048E05E4
:102DD9007E017F08CDCCCD1200038E328F33AE3405
:102DE900AF357411D39F74019E5003022EC4A2F90A
:102DF900B35003022EC1E5354534700375A3D2AE35
:102E090034AF3574016F4E700375A300AE34AF351E
:102E190074026F4E700D9007A6E075F002A4FDAC28
:102E2900F08DA3AE34AF3574036F4E700375A300F4
:102E3900AE34AF3574046F4E700375A300AE34AF72
:102E49003574056F4E700375A300AE34AF35740643
:102E59006F4E700375A300AE34AF3574076F4E70B3
:102E69000375A300AE34AF3574086F4E700375A3B4
:102E790000AE34AF357408BE00039F5016AC32ADB6
:102E890033ED2FFFEC3EFE90005C124BDAE5A3F028
:102E990075A300AE34AF35EFB41009EEB401057473
:102EA90014120075AE34AF35EFB41007EEB4010358
:102EB90075F80D7834124C1A022DE7227535007514
:102EC900340075F809AE34AF357417BE0004D39FCA
:102ED9005003022F9DA2F9B35003022F9AE53545FD
:102EE90034700375A3D2AE34AF3574016F4E7003DD
:102EF90075A300AE34AF3574026F4E700D9007A6FE
:102F0900E075F002A4FDACF08DA3AE34AF357403C7
:102F19006F4E700375A300AE34AF3574046F4E70F5
:102F29000375A300AE34AF3574056F4E700375A3F6
:102F390000AE34AF3574066F4E700375A300AE341E
:102F4900AF3574076F4E700375A300AE34AF357497
:102F5900086F4E700375A300AE34AF357408BE0018
:102F6900039F500C900046124BDAE5A3F075A300BD
:102F7900AE34AF3574166F4E70057414120075AE09
:102F890034AF3574166F4E700375F80D7834124CE2
:102F99001A022ECE22900032E0B4AB028003023036
:102FA9003875350075340075F809AE34AF357412CB
:102FB900BE007CD39F4078A2F9B34070E535453413
:102FC900700375A382AE34AF3574016F4E7003750B
:102FD900A300AE34AF3574026F4E700D9007A6E0B2
:102FE90075F002A4FDACF08DA3AE34AF3574036F58
:102FF9004E700375A300AE34AF357403BE00039F52
:10300900500990004B124BDAE0F5A3AE34AF35749A
:10301900116F4E70057414120075AE34AF3574110A
:103029006F4E700375F80D7834124C1A022FB322C3
:1030390090003BE4F074649007A5F8E4F0E8A3F08D
:10304900122EC574C89007A5F8E4F0E8A3F0900023
:1030590052E0B4371A90004FE0900046F0900050CB
:10306900E0900047F0900051E0900048F0804690D1
:10307900003B7401F074659007A5F8E4F0E8A3F04B
:10308900122EC574C89007A5F8E4F0E8A3F09000E3
:1030990052E0B4371A90004FE0900046F09000508B
:1030A900E0900047F0900051E0900048F0800674ED
:1030B9000290003BF090003CE4F074669007A5F89C
:1030C900E4F0E8A3F0122EC574C89007A5F8E4F05F
:1030D900E8A3F0900051E0B4371290004FE090005F
:1030E90040F0900050E0900049F0807690003C74E8
:1030F90001F074679007A5F8E4F0E8A3F0122EC573
:1031090074C89007A5F8E4F0E8A3F0900051E0B482
:10311900371290004FE0900040F0900050E090008E
:1031290049F0803E740290003CF074689007A5F85D
:10313900E4F0E8A3F0122EC574C89007A5F8E4F0EE
:10314900E8A3F0900051E0B4371290004FE09000EE
:1031590040F0900050E0900049F080067403900020
:103169003CF022E55C2533FFAE3250010E9000653C
:10317900124BDAE0F55DE55C2533FFAE3250010E06
:103189000FBF00010E900065124BDAE0F55E856411
:1031990060E55DB55E05855D5C8041E55ED3955D65
:1031A900401DE55EC3955D855FF0A4FFAEF0E56067
:1031B9008E048F05FF120085ED255DF55C801DE508
:1031C9005DC3955E855FF0A4FFAEF0E5608E048F68
:1031D90005FF120085EDF404255DF55C22E55ED35B
:1031E900955D401DE55EC3955D855FF0A4FFAEF07A
:1031F900E5608E048F05FF120085ED255DF55C8085
:103209001DE55DC3955E855FF0A4FFAEF0E5608EB8
:10321900048F05FF120085EDF404255DF55C22E5B8
:103229003775F00484FF7E008F5CE53775F0048400
:10323900ADF07C008D5F756404753201753300E56E
:103249005CC3943F500512316C80069001A4E0F5EF
:103259005C855C52755100900037E075F020A4FF41
:10326900AEF09000B6E08E048F05FF1200858D5CEC
:1032790090009EE0D39537500302332E9000C2E0B0
:10328900D395374010ED9001A5124BEFE0F5547539
:10329900530002332B90008DE0D395374043E55C12
:1032A9009001A5124BEFE0F55DE55C9001C5124B6D
:1032B900EFE0F55E9000C2E0F4042537F55F900079
:1032C9008DE0FE9000C2E0F4042EF560E55DB55E88
:1032D90005855D5C80031231E6855C547553008079
:1032E90041E55C9001C5124BEFE0F55DE55C9001AD
:1032F900E5124BEFE0F55E90008DE0F4042537F51B
:103309005F90009EE0FE90008DE0F4042EF560E5EC
:103319005DB55E05855D5C80031231E6855C54759B
:1033290053000233D59000C5E0D395375011E55CC1
:10333900900225124BEFE0F5547553000233D590F6
:10334900008EE0D395375043E55C900205124BEFB0
:10335900E0F55DE55C900225124BEFE0F55E90002B
:103369008EE0F4042537F55F9000C5E0FE90008EED
:10337900E0F4042EF560E55DB55E05855D5C8003CE
:103389001231E6855C547553008041E55C9001E596
:10339900124BEFE0F55DE55C900205124BEFE0F5AD
:1033A9005E90009EE0F4042537F55F90008EE0FE04
:1033B90090009EE0F4042EF560E55DB55E05855D3F
:1033C9005C80031231E6855C54755300229000D667
:1033D900E0F561756411753202753300AE24AF25CD
:1033E900E56175F00FA4FDACF0EDD39FEC9E402193
:1033F900E5618E048F05FF120085ED75F010A4FFBD
:10340900AEF0E53775F01184FD7C00ED2FF5628093
:103419000EE53775F01184FF7E00EF24F0F5628523
:10342900625CE53775F01184AFF07E008F5F123171
:103439006C855C63AE24AF259000D6E075F00FA4CF
:10344900FDACF0EDD39FEC9E402875320275331028
:1034590085625C12316C85635D855C5EAE24AF2547
:10346900E5618E048F05FF124BCE8D5F8561601279
:1034790031E6855C5275510075546475530022908C
:1034890000D6E0F561756411753202753300AE241A
:10349900AF25E56175F00FA4FDACF0EDD39FEC9E6F
:1034A9004021E5618E048F05FF120085ED75F0104E
:1034B900A4FFAEF0E53975F01184FD7C00ED2FF520
:1034C90062800EE53975F01184FF7E00EF24F0F576
:1034D9006285625CE53975F01184AFF07E008F5F1B
:1034E90012316C855C63AE24AF259000D6E075F08F
:1034F9000FA4FDACF0EDD39FEC9E40287532027508
:10350900331085625C12316C85635D855C5EAE2427
:10351900AF25E5618E048F05FF124BCE8D5F856166
:10352900601231E6855C527551009000A0E0B40448
:1035390053E53775F00484FF7E008F5CE53775F03D
:103549000484ADF07C008D5F7564047532017533B8
:1035590000E55CC3943F500512316C80069001A4CC
:10356900E0F55CAE51AF52E55C124BB374648E0466
:103579008F05FF120085AE51AF52EF2DFDEE3CFCD9
:103589008C518D527554647553002290006BE0B4D0
:103599000146E53F75F00584FF7E008F5CE53F75C8
:1035A900F00584ADF07C008D5F7564057532057595
:1035B9003300E55CC39417500512316C8006900501
:1035C9007CE0F55CAE53AF54E55C2FFF50010E74FF
:1035D90064124C0A8E538F5490006CE0B40146E596
:1035E9004075F00584FF7E008F5CE54075F0058429
:1035F900ADF07C008D5F756405753205753348E55E
:103609005CC39417500512316C80069005C4E0F52F
:103619005CAE53AF54E55C2FFF50010E7464124C3D
:103629000A8E538F5490007BE0B40249E542C3945B
:103639004175F00584FF7E008F5CE54275F00584D5
:10364900ADF07C008D5F756405753206753300E554
:103659005CC39413500512316C8006900678E0F52E
:103669005CAE53AF54E55C2FFF50010E7464124CED
:103679000A8E538F549000BDE0B4020280030237D2
:1036890033E53775F01584FF7E008F5CE53775F0FB
:103699001584ADF07C008D5F756415753203753343
:1036A900F4E55CC3940B500512316C8006900464F8
:1036B900E0F55CE55C75F0FFA4FFAEF09000BEE0BC
:1036C9008E048F05FF120085ED900060F0E53E75D0
:1036D900F078A4FFAEF074FF8E048F05FF12008509
:1036E9008C328D3374028C068D07124BA58F5CAC1E
:1036F90032AD337404FF124BCE8D5F75640475329D
:103709000675336EE55CC3941D500512316C800655
:103719009006F0E0F55CAE53AF54E55C2FFF500125
:103729000E7464124C0A8E538F5422900073E0B4C5
:1037390001179007AAE02554FFAE5350010E9000DF
:10374900C7E0124C0A8E538F54900073E0B40316ED
:10375900A201B3B3501090005FE0C39405A824B848
:103769000006952540028010900095E02554FFAE93
:103779005350010E8E538F5490006DE0B4020280B5
:1037890003023961900070E0602FE53FD3941E4039
:1037990028900010E0FEA3E0FF9000ABE075F00375
:1037A900A4FDACF0EFD39DEE9C400E9000CFE0A8B5
:1037B90024B80005D3952550030239619000B8E07B
:1037C9008537F0A4FFAEF07405124BB37407124BA2
:1037D900A58E328F33900077E0A824B80004952590
:1037E9005012900078E075F002A4FDACF0EFC39D93
:1037F900EE9C4003023961E53775F00B84FF7E00CA
:103809009005F5124BDAFEE0FFEE90006FE0FEEF57
:103819008E0088F0A4FFAEF074648E048F05FF1249
:1038290000858C328D33900037E075F018A4FFAE17
:10383900F09000B6E08E048F05FF1200858C068D8E
:103849000790060D124BDAAE32AF33E0124BB37468
:10385900648E048F05FF1200858C328D33E53DA8F7
:1038690032B80077D395334072E53DC39533FFE411
:103879009532FE8E328F337428BE00039F500C752B
:103889003328753200740D90003AF0AE32AF3390A0
:103899000070E0124BB374288E048F05FF12008567
:1038A9008C328D33AE51AF52740A8E048F05FF12DC
:1038B90000858D068C07AC32AD33CFCECF12000315
:1038C900740A8E048F05FF1200858C328D33AE5138
:1038D900AF52124C128E518F52807DE53DA832B8FD
:1038E900000495335072AE32AF33E53D124C0A8E67
:1038F900328F337428BE00039F500C7533287532FC
:1039090000740D90003AF0AE32AF33900070E012BF
:103919004BB374288E048F05FF1200858C328D33CA
:10392900AE51AF52740A8E048F05FF1200858D06C1
:103939008C07AC32AD33CFCECF120003740A8E049C
:103949008F05FF1200858C328D33AE51AF52EF2DAA
:10395900FDEE3CFC8C518D5222AE51AF52AC53ADB1
:103969005412000374648E048F05FF1200858C5174
:103979008D52900068E08C068D07124BB374648EEB
:10398900048F05FF1200858C518D52A2084017AE95
:1039990024AF257405BE00039F5002D208E539D330
:1039A90094CC4002D2029000CAE0B402089000CC44
:1039B900E0640160028017AE51AF52E543124BB388
:1039C90074E78E048F05FF1200858C518D5290008B
:1039D9008AE05402601B900081E0A824B80012D349
:1039E9009525400DA208B3B35007E539C3949A4011
:1039F900028028AE5AAF5B90007FE075F002A4FD0B
:103A0900ACF0EF2DFDEE3CFC74022DFD50010CE5F0
:103A190039BC0007D39D400375680185395B755A28
:103A290000E5687003023AB89000DDE0C39568408C
:103A390070E53F75F00584FF7E00900565124BDA4D
:103A4900E0F533753200AE32AF3390008FE0124BA0
:103A5900B374648E048F05FF1200858C348D359004
:103A690000DDE004C395688C068D07124BB3900006
:103A7900DDE08E048F05FF1200858C348D359000B2
:103A890080E08C068D07124BB3740A8E048F05FFF4
:103A9900120085AE51AF52EF2DFDEE3CFC8C518DDD
:103AA9005205689000DDE0C3956850037568009081
:103AB900008AE05401601B90007EE0A824B800123F
:103AC900D39525400DA208B3B35007E537C394CC6D
:103AD9004002802590007CE075F003A4FFAEF0E57C
:103AE900652FFF50010E74032FFF50010EE537BEFD
:103AF9000007D39F4003756901853765E569700340
:103B0900023B939000DEE0C395694070E53F75F094
:103B19000584FF7E00900565124BDAE0F5337532B6
:103B290000AE32AF3390008FE0124BB374648E0451
:103B39008F05FF1200858C348D359000DEE004C3BB
:103B490095698C068D07124BB39000DEE08E048FC9
:103B590005FF1200858C348D3590007DE08C068D33
:103B690007124BB3740A8E048F05FF120085AE51FC
:103B7900AF52EF2DFDEE3CFC8C518D520569900042
:103B8900DEE0C39569500375690090008FE0A85184
:103B9900B800049552500990008FE0F55275510014
:103BA900229000CBE0B401028003023CB5A208B325
:103BB9005003023CB3900096E0B40168AE51AF5295
:103BC900AC24AD25120003743C8E048F05FF12004E
:103BD900859000A6E0BC00109D400D9000A8E0A8CB
:103BE90051B8000495525002D203AE51AF52AC24E1
:103BF900AD25120003743C8E048F05FF12008590D9
:103C090000A6E0C3940ABC0015D39D40119000A8FA
:103C1900E0C39405A851B80005D39552500280021B
:103C2900C2038068AE51AF52AC24AD2512000374B3
:103C3900788E048F05FF1200859000A6E0BC001065
:103C49009D400D9000A8E0A851B800049552500479
:103C5900D2038038AE51AF52AC24AD2512000374A3
:103C6900788E048F05FF1200859000A6E0C3940AA0
:103C7900BC0015D39D40119000A8E0C39405A8513C
:103C8900B80005D3955250028002C203A203B34083
:103C990019AE51AF529000A7E0124BB374648E0471
:103CA9008F05FF1200858C518D528002C20390004E
:103CB900CBE0B40258E53775F00884FF7E008F5CCD
:103CC900E53775F00884ADF07C008D5F7564087583
:103CD90032017533E0E55CC3943F500512316C80C5
:103CE90006900264E0F55CE55C75F05EA4FFAEF059
:103CF900740A8E048F05FF1200858C558D56740247
:103D0900BC000AD39D4006755602755500A200B342
:103D19004006A202B3B35009900016E4F0A3F08064
:103D290024AE51AF527400D39F74019E400C900091
:103D390016E551F0A3E552F0800B74FF900016F8D8
:103D4900E4F0E8A3F09000ADE0D394024006A208A5
:103D5900B3B34002800DAE51AF527402124BB38E11
:103D6900518F52900096E0B4010DAE51AF527402DA
:103D7900124BB38E518F52AE51AF52745E124BB388
:103D8900740A8E048F05FF1200858C518D527402BE
:103D9900BC000AD39D40067552027551009000146B
:103DA900E551F0A3E552F022900037E09003651247
:103DB9004BEFE0F566756764900037E0FE9000A16F
:103DC900E0D39E4037E53775F00884FF7E008F5CAD
:103DD900E53775F00884ADF07C008D5F7564087572
:103DE9003203753396E55CC3941F500512316C801C
:103DF9000690041AE0F55C855C678035E53775F057
:103E09000884FF7E008F5CE53775F00884ADF07C8F
:103E1900008D5F7564087532037533B6E55CC3942C
:103E29001F500512316C800690043AE0F55C855C00
:103E390067229000D7E0F561756411753204753316
:103E490000AE24AF25E56175F00FA4FDACF0EDD30C
:103E59009FEC9E4021E5618E048F05FF120085EDE0
:103E690075F010A4FFAEF0E53775F01184FD7C0004
:103E7900ED2FF562800EE53775F01184FF7E00EFB6
:103E890024F0F56285625CE53775F01184AFF07E48
:103E9900008F5F12316C855C63AE24AF259000D72B
:103EA900E075F00FA4FDACF0EDD39FEC9E402875B2
:103EB900320475331085625C12316C85635D855CF3
:103EC9005EAE24AF25E5618E048F05FF124BCE8DC2
:103ED9005F8561601231E6855C66756764229000D2
:103EE900D7E0F561756411753204753300AE24AFFE
:103EF90025E56175F00FA4FDACF0EDD39FEC9E4074
:103F090021E5618E048F05FF120085ED75F010A47F
:103F1900FFAEF0E53975F01184FD7C00ED2FF562F7
:103F2900800EE53975F01184FF7E00EF24F0F5620B
:103F390085625CE53975F01184AFF07E008F5F1200
:103F4900316C855C63AE24AF259000D7E075F00F26
:103F5900A4FDACF0EDD39FEC9E4028753204753377
:103F69001085625C12316C85635D855C5EAE24AF41
:103F790025E5618E048F05FF124BCE8D5F8561604B
:103F89001231E6855C667567649000D2E0B4047905
:103F9900900037E0FE9000A1E0D39E4037E53775E9
:103FA900F00884FF7E008F5CE53775F00884ADF07A
:103FB9007C008D5F756408753203753396E55CC3C3
:103FC900941F500512316C800690041AE0F55C8547
:103FD9005C678035E53775F00884FF7E008F5CE506
:103FE9003775F00884ADF07C008D5F756408753213
:103FF900037533B6E55CC3941F500512316C800616
:1040090090043AE0F55C855C672290006BE0B401AE
:104019003BE53F75F00584FF7E008F5CE53F75F059
:104029000584ADF07C008D5F7564057532057533C7
:1040390018E55CC39417500512316C8006900594FD
:10404900E0F55CE567255CC39464F56790006CE076
:10405900B4013BE54075F00584FF7E008F5CE540C7
:1040690075F00584ADF07C008D5F756405753205CA
:10407900753360E55CC39417500512316C80069066
:1040890005DCE0F55CE567255CC39464F567E566E6
:104099002567F559900073E0B402109007A9E0254F
:1040A90059FE9000C7E0F4042EF5599000CAE0D3F8
:1040B90094014040E543C394E7501D74E7C3954319
:1040C900FE9007ABE08E00F5F0E884FF7E008F5C80
:1040D900E559255CF559801CE543C394E7FE900733
:1040E900ABE08E00F5F0E884FF7E008F5CE559C3F4
:1040F900955CF559A2084006E5662464F559E55929
:10410900D394644009E559C39464F55980037559FA
:10411900009000A3E0C3955950069000A3E0F5591B
:1041290022D2009000B9E0A824B800049525503B9C
:104139009000B9E0A824B800049525500375590FDB
:104149009000B9E004A824B80004952550037559D6
:104159000A9000B9E02402A824B800049525500566
:10416900755905C200740990003AF07E017F0090EC
:1041790000A9E0124BB39000B8E08E048F05FF123E
:104189000085E537BC000CD39D4008C200740A9035
:10419900003AF09000AAE0C3953F500D9000BCE0B2
:1041A900A824B80006952540028008C200740B9027
:1041B900003AF0A2004003755905900073E0B4037A
:1041C90006A201B3B34002802B90005FE0C39405BF
:1041D900A824B800049525500C900094E0F5597472
:1041E9000C90003AF090005FE0A824B800049525EF
:1041F9005002C200855944900065E02559FE90009F
:1042090037E075F01E84FC7F00EE2CF559229000F2
:1042190037E075F00584FF7E008F5C900037E0750C
:10422900F00584ADF07C008D5F756405753203750A
:1042390033D69000B6E01475F00584FF7E00E55C86
:10424900BE00039F500512316C800BE55C90043B66
:10425900124BEFE0F55CE55C9007ACF09007ACE041
:10426900FE9000A5E0C39E50089000A5E09007AC21
:10427900F022E53F75F00584FF7E00900565124B3D
:10428900DAE0F56BE56BD394644010E56BC3946495
:1042990075F00F84FF7E008F6B8003756B009000B3
:1042A90088E0256BF56B2290079FE0FEA3E0FF7481
:1042B90004124BA5E537124BB3740F8E048F05FF1B
:1042C90012008590079DECF0A3EDF090007BE0B41F
:1042D9000262E542C3944175F00584FF7E008F5C5C
:1042E900E54275F00584ADF07C008D5F7564057558
:1042F9003206753314E55CC39417500512316C808E
:104309000690068CE0F55C90079DE0FEA3E0FF7443
:104319000A8E048F05FF120085E55C8C068D071255
:104329004BB3740A8E048F05FF12008590079DEC2C
:10433900F0A3EDF090079DE0FEA3E0FF9007A3E056
:10434900FCA3E0FDEDD39FEC9E400F9007A3E0F89E
:10435900A3E090079DC8F0A3C8F022900082E0B4C2
:10436900010385254F900082E0B402129000B8E065
:104379008537F0A4FFAEF07408124BA58F4F90005B
:1043890082E0B4030385394F900082E0B4040385C9
:104399003F4F900082E0B40507E540C39414F54F00
:1043A900900082E0B4060385414F900082E0B40793
:1043B9000385424F900082E0B4080385434F900083
:1043C90082E0B40903853E4F900083E0FE900084AB
:1043D900E0D39E404B900082E0B40418900084E042
:1043E900C3954F5002D204900083E0D3954F400209
:1043F900C204802A900083E0C3954F50099000843D
:10440900E0D3954F50028002D204900083E0D39507
:104419004F5009900084E0C3954F5002C204802A8E
:10442900900083E0D3954F4009900084E0C3954FF5
:1044390040028002C204900083E0C3954F40099076
:104449000084E0D3954F4002D20422900085E0B465
:10445900010385254F900085E0B402129000B8E071
:104469008537F0A4FFAEF07408124BA58F4F90006A
:1044790085E0B4030385394F900085E0B4040385D2
:104489003F4F900085E0B40507E540C39414F54F0C
:10449900900085E0B4060385414F900085E0B4079C
:1044A9000385424F900085E0B4080385434F90008F
:1044B90085E0B40903853E4F900086E0FE900087B1
:1044C900E0D39E4040900086E0C3954F500990008C
:1044D90087E0D3954F50028002D206900086E0D340
:1044E900954F5009900087E0C3954F5002C206903E
:1044F9000085E0B401099000C4E0D39539500280E9
:1045090002C206802A900086E0D3954F40099000A8
:1045190087E0C3954F40028002C206900086E0C33F
:10452900954F4009900087E0D3954F4002D206226B
:10453900AE57AF5874F5D39F74019E40087857124F
:104549004C1A024634755801755700AE24AF25E55B
:104559006BBE000DD39F400990009AE0D3956C4043
:1045690002801B756C00E56BC39525F54F90009D86
:10457900E0D3956A4006E56A254FF56A8002056C25
:10458900900076E0D39539401CE537C3953840153E
:10459900AE24AF25E56BBE00039F500990009BE058
:1045A900D3956D400280579007ADE0A824B8000468
:1045B90095255003756F009007ADE0A824B8000B4E
:1045C900D395254006E5259007ADF0E56F702AE5FE
:1045D90025C3956BF54FE54FD394054003754F05FA
:1045E90090009CE0C3956A5007E54FC3956A400265
:1045F9008007E56AC3954FF56A756D008002056D00
:10460900E56F7016900076E0C39539500DE56B247F
:1046190005A824B8000695254002800F900089E07E
:10462900F56A756F0174789007ADF022AE57AF58EF
:1046390074E9D39F74039E40087857124C1A0247B5
:10464900E2755801755700756A32A21D402A756ACC
:1046590019900089E075F002A4FFAEF0E56CBE0088
:1046690006D39F4002D21D056C756F0374789007BD
:10467900ADF0756E000247D1AE24AF25E56B6F4EE4
:1046890070030247D1E56BBE000DD39F400990002E
:104699009AE0D3956C40028017756C00A208B3B3F9
:1046A9005007E56FC3940340028003756A19800DB2
:1046B900E56BC39525F54FE56C254FF56C900076B4
:1046C900E0D39539400E9007ADE0A824B80007D390
:1046D90095254002800C056E900089E0B56E037542
:1046E9006F00E56FB4030DE56B2402A824B800063A
:1046F90095254002800A056EE56EB43C03756F028C
:10470900E56FB402299007ADE0A824B8000ED3954F
:10471900254009E5259007ADF0756E00900076E01B
:10472900C395395009756E0074789007ADF0E56F3F
:10473900705A900076E0D39539401CE537D3953807
:104749004015AE24AF25E56BBE00039F50099000CC
:104759009BE0D3956D40028008756D00756A4B80AA
:1047690028E525C3956BF54FE54FD39405400375AF
:104779004F05900076E0D395394008E56D254FF552
:104789006D8006E56D2406F56D756E00E56F701692
:10479900900076E0C39539500DE56B2405A824B83F
:1047A9000006952540028003756F01E56FB4011875
:1047B900756A19056E900089E0B56E06756F027508
:1047C9006E0074789007ADF0E56A75F00AA4FFAE43
:0A47D900F09007A7EEF0A3EFF02226
:094BEF002582F5825002058322A3
:0F4B960025E050020583258250020583F5822217
:10006400EF2F500205832582F582E5833E2EF5832A
:010074002269
:104C0A00CFC39FFF50011E22C3EF9DFFEE9CFE22E1
:094BF800E493F608740193F6221F
:084C1A000806B600021806228C
:0D4BC100A3E004F07006124BE5E004F022C2
:0E003900A3E014F0B4FF06124BE5E014F02231
:0E4BA500048007C3CE13CECF13CFD5E0F62287
:104AB500BC000FBE0008ED8FF084FFADF022E4FED0
:104AC500FF22BE000DEF60FE54F0606F20E7030289
:104AD5004B6BEAC0E0EBC0E078017A0075F001EEBF
:104AE50020E710EF25E0FFEE33FE0AC5F023C5F001
:104AF50030E7F0EA5407F9096A7A007B006001089B
:104B0500C3EC9E40167004ED9F4010ED9FFDEC9E9A
:104B1500FCE5F0CA4ACA03F5F08005E5F003F5F0B7
:104B2500C3EE13FEEF13FFD9D77908CACBCAD8D085
:104B3500EAFEEBFFD0E0FBD0E0FA22EC8FF084FC3C
:104B4500ED54F045F0C48FF084FEEDC454F045F00B
:104B5500C48FF084FDEEC4FE54F02DFFEE540F3CDF
:104B6500FEADF07C0022790078008FF0EC7E082005
:104B7500E70DC3CD33CD33C933C9C833C8DEF0849F
:104B850049F9E5F08FF0BE00E6FD7C00E9FFE8FE9F
:014B950022FD
:0E4BB300F88FF0A4FFE5F0CE88F0A42EFE22CD
:10000300EF8DF0A4F9A8F0EF8CF0A428F8EE8DF0B2
:06001300A428FEE9FF2213
:10007500600D782B02007F007830D8FED5E0F8229D
:10008500EEC0E07E00124AB5EFFDEEFCD0E0FE22A8
:0C4BCE00EEC0E07E00124AB5D0E0FE22EE
:03001B0002001EC2
:03009B0002004917
:03000000024C01AE
:094C010075817075D00002066B8C
:104BDA00E5822FF582E5833EF583220582D582029E
:054BEA00158315822275
:10001E00C0E0C0F0C083C082C0D075D000120616FA
:0B002E00D0D0D082D083D0F0D0E032E0
:10004900C0E0C0F0C083C082C0D075D000120619CC
:0B005900D0D0D082D083D0F0D0E032B5
:00000001FF
